
 Start         Length     Name                   Class
 0001:00000000 00006348H .text                   CODE
 0002:00000000 0000012CH .data                   DATA
 0002:0000012C 00000075H .bss                    BSS


Detailed map of segments

 0001:00000000 00000196 C=CODE     S=.text    G=(none)   M=System   ACBP=A9
 0001:00000198 000001EC C=CODE     S=.text    G=(none)   M=SysInit  ACBP=A9
 0001:00000384 00000050 C=CODE     S=.text    G=(none)   M=Windows  ACBP=A9
 0001:000003D4 0000000E C=CODE     S=.text    G=(none)   M=Types    ACBP=A9
 0001:000003E4 00000038 C=CODE     S=.text    G=(none)   M=Messages ACBP=A9
 0001:0000041C 0000000E C=CODE     S=.text    G=(none)   M=ActiveX  ACBP=A9
 0001:0000042C 0000004E C=CODE     S=.text    G=(none)   M=SysUtils ACBP=A9
 0001:0000047C 0000000E C=CODE     S=.text    G=(none)   M=SysConst ACBP=A9
 0001:0000048C 00000106 C=CODE     S=.text    G=(none)   M=Classes  ACBP=A9
 0001:00000594 0000000E C=CODE     S=.text    G=(none)   M=TypInfo  ACBP=A9
 0001:000005A4 0000000E C=CODE     S=.text    G=(none)   M=Variants ACBP=A9
 0001:000005B4 0000000E C=CODE     S=.text    G=(none)   M=VarUtils ACBP=A9
 0001:000005C4 0000000E C=CODE     S=.text    G=(none)   M=RTLConsts ACBP=A9
 0001:000005D4 00000036 C=CODE     S=.text    G=(none)   M=Graphics ACBP=A9
 0001:0000060C 0000000E C=CODE     S=.text    G=(none)   M=Consts   ACBP=A9
 0001:0000061C 000000E6 C=CODE     S=.text    G=(none)   M=Controls ACBP=A9
 0001:00000704 0000002E C=CODE     S=.text    G=(none)   M=ActnList ACBP=A9
 0001:00000734 0000000E C=CODE     S=.text    G=(none)   M=Contnrs  ACBP=A9
 0001:00000744 0000000E C=CODE     S=.text    G=(none)   M=Math     ACBP=A9
 0001:00000754 0000000E C=CODE     S=.text    G=(none)   M=ImgList  ACBP=A9
 0001:00000764 00000038 C=CODE     S=.text    G=(none)   M=CommCtrl ACBP=A9
 0001:0000079C 00000116 C=CODE     S=.text    G=(none)   M=Forms    ACBP=A9
 0001:000008B4 0000000E C=CODE     S=.text    G=(none)   M=HelpIntfs ACBP=A9
 0001:000008C4 0000000E C=CODE     S=.text    G=(none)   M=MultiMon ACBP=A9
 0001:000008D4 00000038 C=CODE     S=.text    G=(none)   M=Imm      ACBP=A9
 0001:0000090C 00000026 C=CODE     S=.text    G=(none)   M=Menus    ACBP=A9
 0001:00000934 0000000E C=CODE     S=.text    G=(none)   M=Themes   ACBP=A9
 0001:00000944 0000000E C=CODE     S=.text    G=(none)   M=UxTheme  ACBP=A9
 0001:00000954 0000000E C=CODE     S=.text    G=(none)   M=SyncObjs ACBP=A9
 0001:00000964 00000016 C=CODE     S=.text    G=(none)   M=ComCtrls ACBP=A9
 0001:0000097C 00000038 C=CODE     S=.text    G=(none)   M=ShlObj   ACBP=A9
 0001:000009B4 00000038 C=CODE     S=.text    G=(none)   M=UrlMon   ACBP=A9
 0001:000009EC 00000038 C=CODE     S=.text    G=(none)   M=WinInet  ACBP=A9
 0001:00000A24 00000038 C=CODE     S=.text    G=(none)   M=RegStr   ACBP=A9
 0001:00000A5C 00000040 C=CODE     S=.text    G=(none)   M=ShellAPI ACBP=A9
 0001:00000A9C 0000000E C=CODE     S=.text    G=(none)   M=ListActns ACBP=A9
 0001:00000AAC 0000000E C=CODE     S=.text    G=(none)   M=ExtCtrls ACBP=A9
 0001:00000ABC 0000001E C=CODE     S=.text    G=(none)   M=StdCtrls ACBP=A9
 0001:00000ADC 0000000E C=CODE     S=.text    G=(none)   M=WinHelpViewer ACBP=A9
 0001:00000AEC 0000000E C=CODE     S=.text    G=(none)   M=StdActns ACBP=A9
 0001:00000AFC 00000016 C=CODE     S=.text    G=(none)   M=Dialogs  ACBP=A9
 0001:00000B14 0000000E C=CODE     S=.text    G=(none)   M=Printers ACBP=A9
 0001:00000B24 00000038 C=CODE     S=.text    G=(none)   M=WinSpool ACBP=A9
 0001:00000B5C 00000038 C=CODE     S=.text    G=(none)   M=CommDlg  ACBP=A9
 0001:00000B94 00000038 C=CODE     S=.text    G=(none)   M=Dlgs     ACBP=A9
 0001:00000BCC 0000000E C=CODE     S=.text    G=(none)   M=StrUtils ACBP=A9
 0001:00000BDC 0000001E C=CODE     S=.text    G=(none)   M=Clipbrd  ACBP=A9
 0001:00000BFC 0000000E C=CODE     S=.text    G=(none)   M=FlatSB   ACBP=A9
 0001:00000C0C 0000000E C=CODE     S=.text    G=(none)   M=ToolWin  ACBP=A9
 0001:00000C1C 00000038 C=CODE     S=.text    G=(none)   M=RichEdit ACBP=A9
 0001:00000C54 0000000E C=CODE     S=.text    G=(none)   M=ExtActns ACBP=A9
 0001:00000C64 0000000E C=CODE     S=.text    G=(none)   M=Registry ACBP=A9
 0001:00000C74 00000016 C=CODE     S=.text    G=(none)   M=IniFiles ACBP=A9
 0001:00000C8C 0000000E C=CODE     S=.text    G=(none)   M=ExtDlgs  ACBP=A9
 0001:00000C9C 0000000E C=CODE     S=.text    G=(none)   M=Buttons  ACBP=A9
 0001:00000CAC 0000000E C=CODE     S=.text    G=(none)   M=Mapi     ACBP=A9
 0001:00000CBC 0000000E C=CODE     S=.text    G=(none)   M=ComStrs  ACBP=A9
 0001:00000CCC 0000004E C=CODE     S=.text    G=(none)   M=DockForm ACBP=A9
 0001:00000D1C 0000000E C=CODE     S=.text    G=(none)   M=IDEMessages ACBP=A9
 0001:00000D2C 0000004E C=CODE     S=.text    G=(none)   M=DeskForm ACBP=A9
 0001:00000D7C 0000000E C=CODE     S=.text    G=(none)   M=DesignIntf ACBP=A9
 0001:00000D8C 0000000E C=CODE     S=.text    G=(none)   M=DesignMenus ACBP=A9
 0001:00000D9C 0000001E C=CODE     S=.text    G=(none)   M=DeskUtil ACBP=A9
 0001:00000DBC 0000000E C=CODE     S=.text    G=(none)   M=DeskStrs ACBP=A9
 0001:00000DCC 0000000E C=CODE     S=.text    G=(none)   M=IDEDockPanel ACBP=A9
 0001:00000DDC 0000000E C=CODE     S=.text    G=(none)   M=TabDock  ACBP=A9
 0001:00000DEC 0000000E C=CODE     S=.text    G=(none)   M=JoinDock ACBP=A9
 0001:00000DFC 0000000E C=CODE     S=.text    G=(none)   M=BaseDock ACBP=A9
 0001:00000E0C 0000000E C=CODE     S=.text    G=(none)   M=IDEDockCtrls ACBP=A9
 0001:00000E1C 0000000E C=CODE     S=.text    G=(none)   M=ToolsAPI ACBP=A9
 0001:00000E2C 00000090 C=CODE     S=.text    G=(none)   M=RegExpConst ACBP=A9
 0001:00000EBC 00001CE0 C=CODE     S=.text    G=(none)   M=RegExpComp ACBP=A9
 0001:00002B9C 0000000E C=CODE     S=.text    G=(none)   M=ToolIntf ACBP=A9
 0001:00002BAC 0000000E C=CODE     S=.text    G=(none)   M=FileIntf ACBP=A9
 0001:00002BBC 00000026 C=CODE     S=.text    G=(none)   M=VirtIntf ACBP=A9
 0001:00002BE4 0000000E C=CODE     S=.text    G=(none)   M=EditIntf ACBP=A9
 0001:00002BF4 0000000E C=CODE     S=.text    G=(none)   M=ActnPopup ACBP=A9
 0001:00002C04 0000000E C=CODE     S=.text    G=(none)   M=ActnCtrls ACBP=A9
 0001:00002C14 0000000E C=CODE     S=.text    G=(none)   M=GraphUtil ACBP=A9
 0001:00002C24 0000000E C=CODE     S=.text    G=(none)   M=ActnMan  ACBP=A9
 0001:00002C34 0000000E C=CODE     S=.text    G=(none)   M=ActnColorMaps ACBP=A9
 0001:00002C44 0000000E C=CODE     S=.text    G=(none)   M=ActnMenus ACBP=A9
 0001:00002C54 0000000E C=CODE     S=.text    G=(none)   M=ShadowWnd ACBP=A9
 0001:00002C64 00000038 C=CODE     S=.text    G=(none)   M=MMSystem ACBP=A9
 0001:00002C9C 0000000E C=CODE     S=.text    G=(none)   M=XPActnCtrls ACBP=A9
 0001:00002CAC 00000016 C=CODE     S=.text    G=(none)   M=MsgLines ACBP=A9
 0001:00002CC4 0000000E C=CODE     S=.text    G=(none)   M=ToolUtils ACBP=A9
 0001:00002CD4 0000000E C=CODE     S=.text    G=(none)   M=MsgLinesIntf ACBP=A9
 0001:00002CE4 0000001E C=CODE     S=.text    G=(none)   M=Events   ACBP=A9
 0001:00002D04 0000000E C=CODE     S=.text    G=(none)   M=MsgViewForm ACBP=A9
 0001:00002D14 0000000E C=CODE     S=.text    G=(none)   M=Tabs     ACBP=A9
 0001:00002D24 0000000E C=CODE     S=.text    G=(none)   M=MsgView  ACBP=A9
 0001:00002D34 0000000E C=CODE     S=.text    G=(none)   M=Grids    ACBP=A9
 0001:00002D44 0000000E C=CODE     S=.text    G=(none)   M=Mask     ACBP=A9
 0001:00002D54 0000000E C=CODE     S=.text    G=(none)   M=MaskUtils ACBP=A9
 0001:00002D64 0000000E C=CODE     S=.text    G=(none)   M=AppUtils ACBP=A9
 0001:00002D74 0000000E C=CODE     S=.text    G=(none)   M=VEdTypes ACBP=A9
 0001:00002D84 0000000E C=CODE     S=.text    G=(none)   M=VEdOpts  ACBP=A9
 0001:00002D94 0000000E C=CODE     S=.text    G=(none)   M=EK       ACBP=A9
 0001:00002DA4 0000000E C=CODE     S=.text    G=(none)   M=EdKrnl   ACBP=A9
 0001:00002DB4 0000000E C=CODE     S=.text    G=(none)   M=IDEKbd   ACBP=A9
 0001:00002DC4 0000000E C=CODE     S=.text    G=(none)   M=ComObj   ACBP=A9
 0001:00002DD4 0000000E C=CODE     S=.text    G=(none)   M=ComConst ACBP=A9
 0001:00002DE4 00000016 C=CODE     S=.text    G=(none)   M=KbClient ACBP=A9
 0001:00002DFC 0000000E C=CODE     S=.text    G=(none)   M=IDEServices ACBP=A9
 0001:00002E0C 0000000E C=CODE     S=.text    G=(none)   M=CodeMgr  ACBP=A9
 0001:00002E1C 0000000E C=CODE     S=.text    G=(none)   M=IDEModel ACBP=A9
 0001:00002E2C 0000000E C=CODE     S=.text    G=(none)   M=IDEEvent ACBP=A9
 0001:00002E3C 0000000E C=CODE     S=.text    G=(none)   M=IDEUtil  ACBP=A9
 0001:00002E4C 0000000E C=CODE     S=.text    G=(none)   M=IDEConst ACBP=A9
 0001:00002E5C 0000000E C=CODE     S=.text    G=(none)   M=ResUtils ACBP=A9
 0001:00002E6C 0000000E C=CODE     S=.text    G=(none)   M=OptIntf  ACBP=A9
 0001:00002E7C 0000000E C=CODE     S=.text    G=(none)   M=IDEHistoryManager ACBP=A9
 0001:00002E8C 0000000E C=CODE     S=.text    G=(none)   M=IDERegIniPropSet ACBP=A9
 0001:00002E9C 0000000E C=CODE     S=.text    G=(none)   M=IDEPropSet ACBP=A9
 0001:00002EAC 0000000E C=CODE     S=.text    G=(none)   M=PackageList ACBP=A9
 0001:00002EBC 0000000E C=CODE     S=.text    G=(none)   M=UIUtils  ACBP=A9
 0001:00002ECC 0000000E C=CODE     S=.text    G=(none)   M=VerInf   ACBP=A9
 0001:00002EDC 0000000E C=CODE     S=.text    G=(none)   M=ComTypes ACBP=A9
 0001:00002EEC 0000000E C=CODE     S=.text    G=(none)   M=DbkHelper ACBP=A9
 0001:00002EFC 0000000E C=CODE     S=.text    G=(none)   M=dbk_tlb  ACBP=A9
 0001:00002F0C 0000000E C=CODE     S=.text    G=(none)   M=StdVCL   ACBP=A9
 0001:00002F1C 0000000E C=CODE     S=.text    G=(none)   M=OleCtrls ACBP=A9
 0001:00002F2C 0000000E C=CODE     S=.text    G=(none)   M=AxCtrls  ACBP=A9
 0001:00002F3C 0000000E C=CODE     S=.text    G=(none)   M=OleConst ACBP=A9
 0001:00002F4C 0000000E C=CODE     S=.text    G=(none)   M=IDEVersionInfo ACBP=A9
 0001:00002F5C 0000000E C=CODE     S=.text    G=(none)   M=AppStrs  ACBP=A9
 0001:00002F6C 0000000E C=CODE     S=.text    G=(none)   M=RegistryEx ACBP=A9
 0001:00002F7C 0000000E C=CODE     S=.text    G=(none)   M=AppConst ACBP=A9
 0001:00002F8C 0000000E C=CODE     S=.text    G=(none)   M=FileUtils ACBP=A9
 0001:00002F9C 0000000E C=CODE     S=.text    G=(none)   M=FileCtrl ACBP=A9
 0001:00002FAC 0000000E C=CODE     S=.text    G=(none)   M=EnvVariableFrame ACBP=A9
 0001:00002FBC 0000000E C=CODE     S=.text    G=(none)   M=EnvVariableEntry ACBP=A9
 0001:00002FCC 0000000E C=CODE     S=.text    G=(none)   M=Containers ACBP=A9
 0001:00002FDC 0000000E C=CODE     S=.text    G=(none)   M=MakeObjs ACBP=A9
 0001:00002FEC 0000000E C=CODE     S=.text    G=(none)   M=ProjectMgr ACBP=A9
 0001:00002FFC 0000000E C=CODE     S=.text    G=(none)   M=IDEControl ACBP=A9
 0001:0000300C 0000000E C=CODE     S=.text    G=(none)   M=IDEPeer  ACBP=A9
 0001:0000301C 0000000E C=CODE     S=.text    G=(none)   M=IDEItem  ACBP=A9
 0001:0000302C 0000000E C=CODE     S=.text    G=(none)   M=IDEUIEvent ACBP=A9
 0001:0000303C 0000000E C=CODE     S=.text    G=(none)   M=IDEFixups ACBP=A9
 0001:0000304C 0000000E C=CODE     S=.text    G=(none)   M=IDEMulticast ACBP=A9
 0001:0000305C 0000000E C=CODE     S=.text    G=(none)   M=IDEViewImpl ACBP=A9
 0001:0000306C 0000000E C=CODE     S=.text    G=(none)   M=IDEUtil2 ACBP=A9
 0001:0000307C 0000000E C=CODE     S=.text    G=(none)   M=IDESubfocus ACBP=A9
 0001:0000308C 0000000E C=CODE     S=.text    G=(none)   M=IDESelection ACBP=A9
 0001:0000309C 0000000E C=CODE     S=.text    G=(none)   M=IDEModelEvent ACBP=A9
 0001:000030AC 0000000E C=CODE     S=.text    G=(none)   M=IDEViewManager ACBP=A9
 0001:000030BC 0000000E C=CODE     S=.text    G=(none)   M=IDEView  ACBP=A9
 0001:000030CC 0000000E C=CODE     S=.text    G=(none)   M=IDEItemEditors ACBP=A9
 0001:000030DC 0000000E C=CODE     S=.text    G=(none)   M=IDEItemPainters ACBP=A9
 0001:000030EC 0000000E C=CODE     S=.text    G=(none)   M=IDEGraphImpl ACBP=A9
 0001:000030FC 0000000E C=CODE     S=.text    G=(none)   M=IDEJgl   ACBP=A9
 0001:0000310C 0000000E C=CODE     S=.text    G=(none)   M=IDESelectionImpl ACBP=A9
 0001:0000311C 0000000E C=CODE     S=.text    G=(none)   M=IDESubfocusImpl ACBP=A9
 0001:0000312C 0000000E C=CODE     S=.text    G=(none)   M=IDEModelImpl ACBP=A9
 0001:0000313C 0000000E C=CODE     S=.text    G=(none)   M=IDEVectorImpl ACBP=A9
 0001:0000314C 0000000E C=CODE     S=.text    G=(none)   M=IDESingletonImpl ACBP=A9
 0001:0000315C 0000000E C=CODE     S=.text    G=(none)   M=IDEViewManagerImpl ACBP=A9
 0001:0000316C 0000000E C=CODE     S=.text    G=(none)   M=Modules  ACBP=A9
 0001:0000317C 0000000E C=CODE     S=.text    G=(none)   M=ComponentDesigner ACBP=A9
 0001:0000318C 0000000E C=CODE     S=.text    G=(none)   M=Update   ACBP=A9
 0001:0000319C 0000000E C=CODE     S=.text    G=(none)   M=LibConst ACBP=A9
 0001:000031AC 0000000E C=CODE     S=.text    G=(none)   M=DesignEditors ACBP=A9
 0001:000031BC 0000000E C=CODE     S=.text    G=(none)   M=Proxies  ACBP=A9
 0001:000031CC 0000000E C=CODE     S=.text    G=(none)   M=DesignConst ACBP=A9
 0001:000031DC 0000000E C=CODE     S=.text    G=(none)   M=Designer ACBP=A9
 0001:000031EC 0000000E C=CODE     S=.text    G=(none)   M=StFilSys ACBP=A9
 0001:000031FC 0000000E C=CODE     S=.text    G=(none)   M=IStreams ACBP=A9
 0001:0000320C 0000000E C=CODE     S=.text    G=(none)   M=TopLevels ACBP=A9
 0001:0000321C 0000000E C=CODE     S=.text    G=(none)   M=TreeIntf ACBP=A9
 0001:0000322C 0000000E C=CODE     S=.text    G=(none)   M=EditorViewSupport ACBP=A9
 0001:0000323C 0000000E C=CODE     S=.text    G=(none)   M=CompIntf ACBP=A9
 0001:0000324C 0000000E C=CODE     S=.text    G=(none)   M=ExplorerIntf ACBP=A9
 0001:0000325C 0000000E C=CODE     S=.text    G=(none)   M=Updaters ACBP=A9
 0001:0000326C 0000000E C=CODE     S=.text    G=(none)   M=Symbols  ACBP=A9
 0001:0000327C 0000000E C=CODE     S=.text    G=(none)   M=Context  ACBP=A9
 0001:0000328C 0000000E C=CODE     S=.text    G=(none)   M=ProjectIntf ACBP=A9
 0001:0000329C 0000000E C=CODE     S=.text    G=(none)   M=ComInOut ACBP=A9
 0001:000032AC 0000000E C=CODE     S=.text    G=(none)   M=ComMgr   ACBP=A9
 0001:000032BC 0000000E C=CODE     S=.text    G=(none)   M=TypeLib  ACBP=A9
 0001:000032CC 0000000E C=CODE     S=.text    G=(none)   M=tlberror ACBP=A9
 0001:000032DC 0000000E C=CODE     S=.text    G=(none)   M=TlbConst ACBP=A9
 0001:000032EC 0000000E C=CODE     S=.text    G=(none)   M=regutl   ACBP=A9
 0001:000032FC 0000000E C=CODE     S=.text    G=(none)   M=TlbHash  ACBP=A9
 0001:0000330C 0000000E C=CODE     S=.text    G=(none)   M=tlbdebug ACBP=A9
 0001:0000331C 0000000E C=CODE     S=.text    G=(none)   M=guidutl  ACBP=A9
 0001:0000332C 0000000E C=CODE     S=.text    G=(none)   M=ComPlusUtl ACBP=A9
 0001:0000333C 0000000E C=CODE     S=.text    G=(none)   M=DTLWrite ACBP=A9
 0001:0000334C 0000000E C=CODE     S=.text    G=(none)   M=TlbWrite ACBP=A9
 0001:0000335C 0000000E C=CODE     S=.text    G=(none)   M=TlbUtils ACBP=A9
 0001:0000336C 0000000E C=CODE     S=.text    G=(none)   M=DotNetInterop ACBP=A9
 0001:0000337C 0000000E C=CODE     S=.text    G=(none)   M=AgeCache ACBP=A9
 0001:0000338C 0000000E C=CODE     S=.text    G=(none)   M=StatIntf ACBP=A9
 0001:0000339C 0000000E C=CODE     S=.text    G=(none)   M=Creators ACBP=A9
 0001:000033AC 0000000E C=CODE     S=.text    G=(none)   M=Debug    ACBP=A9
 0001:000033BC 0000000E C=CODE     S=.text    G=(none)   M=PakLoad  ACBP=A9
 0001:000033CC 0000000E C=CODE     S=.text    G=(none)   M=Editors  ACBP=A9
 0001:000033DC 0000000E C=CODE     S=.text    G=(none)   M=XPStyleActnCtrls ACBP=A9
 0001:000033EC 0000000E C=CODE     S=.text    G=(none)   M=IDEMenuAction ACBP=A9
 0001:000033FC 0000000E C=CODE     S=.text    G=(none)   M=IDETabControl ACBP=A9
 0001:0000340C 0000000E C=CODE     S=.text    G=(none)   M=BaseEnvironDialog ACBP=A9
 0001:0000341C 0000000E C=CODE     S=.text    G=(none)   M=IDEPropSheet ACBP=A9
 0001:0000342C 0000000E C=CODE     S=.text    G=(none)   M=EdTrackr ACBP=A9
 0001:0000343C 0000000E C=CODE     S=.text    G=(none)   M=EdProcs  ACBP=A9
 0001:0000344C 0000000E C=CODE     S=.text    G=(none)   M=GenericHighlighter ACBP=A9
 0001:0000345C 0000000E C=CODE     S=.text    G=(none)   M=Highlighters ACBP=A9
 0001:0000346C 0000000E C=CODE     S=.text    G=(none)   M=IniHighlighter ACBP=A9
 0001:0000347C 0000000E C=CODE     S=.text    G=(none)   M=PHPHighlighter ACBP=A9
 0001:0000348C 0000000E C=CODE     S=.text    G=(none)   M=JSHighlighter ACBP=A9
 0001:0000349C 0000000E C=CODE     S=.text    G=(none)   M=EnvOptions ACBP=A9
 0001:000034AC 0000000E C=CODE     S=.text    G=(none)   M=AddInEnvOptions ACBP=A9
 0001:000034BC 0000000E C=CODE     S=.text    G=(none)   M=PakUtil  ACBP=A9
 0001:000034CC 0000000E C=CODE     S=.text    G=(none)   M=DocModul ACBP=A9
 0001:000034DC 0000000E C=CODE     S=.text    G=(none)   M=VirtFile ACBP=A9
 0001:000034EC 0000000E C=CODE     S=.text    G=(none)   M=ToolMain ACBP=A9
 0001:000034FC 0000000E C=CODE     S=.text    G=(none)   M=Gallery  ACBP=A9
 0001:0000350C 0000000E C=CODE     S=.text    G=(none)   M=BaseModExplorerForm ACBP=A9
 0001:0000351C 0000000E C=CODE     S=.text    G=(none)   M=DebugOpts ACBP=A9
 0001:0000352C 0000000E C=CODE     S=.text    G=(none)   M=ExprDlg  ACBP=A9
 0001:0000353C 0000000E C=CODE     S=.text    G=(none)   M=IDEPropCtrls ACBP=A9
 0001:0000354C 0000000E C=CODE     S=.text    G=(none)   M=ColorGrd ACBP=A9
 0001:0000355C 0000000E C=CODE     S=.text    G=(none)   M=CmdConst ACBP=A9
 0001:0000356C 0000000E C=CODE     S=.text    G=(none)   M=MsgWnds  ACBP=A9
 0001:0000357C 0000000E C=CODE     S=.text    G=(none)   M=FileFind ACBP=A9
 0001:0000358C 0000000E C=CODE     S=.text    G=(none)   M=PrintSel ACBP=A9
 0001:0000359C 0000000E C=CODE     S=.text    G=(none)   M=Verify   ACBP=A9
 0001:000035AC 0000000E C=CODE     S=.text    G=(none)   M=ComDebug ACBP=A9
 0001:000035BC 0000000E C=CODE     S=.text    G=(none)   M=EvalMod  ACBP=A9
 0001:000035CC 0000000E C=CODE     S=.text    G=(none)   M=DockToolForm ACBP=A9
 0001:000035DC 0000000E C=CODE     S=.text    G=(none)   M=IDEIntf  ACBP=A9
 0001:000035EC 0000000E C=CODE     S=.text    G=(none)   M=ExptIntf ACBP=A9
 0001:000035FC 0000000E C=CODE     S=.text    G=(none)   M=PkgProjects ACBP=A9
 0001:0000360C 0000000E C=CODE     S=.text    G=(none)   M=Desktop  ACBP=A9
 0001:0000361C 0000000E C=CODE     S=.text    G=(none)   M=ProjectFrm ACBP=A9
 0001:0000362C 0000000E C=CODE     S=.text    G=(none)   M=TreeSearch ACBP=A9
 0001:0000363C 0000000E C=CODE     S=.text    G=(none)   M=PkgEditors ACBP=A9
 0001:0000364C 0000000E C=CODE     S=.text    G=(none)   M=PkgContainers ACBP=A9
 0001:0000365C 0000000E C=CODE     S=.text    G=(none)   M=ContainerSelector ACBP=A9
 0001:0000366C 0000000E C=CODE     S=.text    G=(none)   M=Masks    ACBP=A9
 0001:0000367C 0000000E C=CODE     S=.text    G=(none)   M=CompHelp ACBP=A9
 0001:0000368C 0000000E C=CODE     S=.text    G=(none)   M=HelpSelector ACBP=A9
 0001:0000369C 0000000E C=CODE     S=.text    G=(none)   M=ComPrgrs ACBP=A9
 0001:000036AC 0000000E C=CODE     S=.text    G=(none)   M=Compiler ACBP=A9
 0001:000036BC 0000000E C=CODE     S=.text    G=(none)   M=StandardHighlighters ACBP=A9
 0001:000036CC 0000000E C=CODE     S=.text    G=(none)   M=PackageState ACBP=A9
 0001:000036DC 0000000E C=CODE     S=.text    G=(none)   M=PakMgr   ACBP=A9
 0001:000036EC 0000000E C=CODE     S=.text    G=(none)   M=ExpertReg ACBP=A9
 0001:000036FC 0000000E C=CODE     S=.text    G=(none)   M=CompList ACBP=A9
 0001:0000370C 0000000E C=CODE     S=.text    G=(none)   M=PalMgr   ACBP=A9
 0001:0000371C 0000000E C=CODE     S=.text    G=(none)   M=ViewDlg  ACBP=A9
 0001:0000372C 0000000E C=CODE     S=.text    G=(none)   M=Palettes ACBP=A9
 0001:0000373C 0000000E C=CODE     S=.text    G=(none)   M=PakWarn  ACBP=A9
 0001:0000374C 0000000E C=CODE     S=.text    G=(none)   M=AddRequires ACBP=A9
 0001:0000375C 0000000E C=CODE     S=.text    G=(none)   M=AddContainsRequiresBase ACBP=A9
 0001:0000376C 0000000E C=CODE     S=.text    G=(none)   M=PackageAddBase ACBP=A9
 0001:0000377C 0000000E C=CODE     S=.text    G=(none)   M=AddContains ACBP=A9
 0001:0000378C 0000000E C=CODE     S=.text    G=(none)   M=AddContainsRequires ACBP=A9
 0001:0000379C 0000000E C=CODE     S=.text    G=(none)   M=PakAnaly ACBP=A9
 0001:000037AC 0000000E C=CODE     S=.text    G=(none)   M=PakList  ACBP=A9
 0001:000037BC 0000000E C=CODE     S=.text    G=(none)   M=CheckLst ACBP=A9
 0001:000037CC 0000000E C=CODE     S=.text    G=(none)   M=PakRemRu ACBP=A9
 0001:000037DC 0000000E C=CODE     S=.text    G=(none)   M=InstColl ACBP=A9
 0001:000037EC 0000000E C=CODE     S=.text    G=(none)   M=Archiver ACBP=A9
 0001:000037FC 0000000E C=CODE     S=.text    G=(none)   M=ZLib     ACBP=A9
 0001:0000380C 0000000E C=CODE     S=.text    G=(none)   M=ZLibConst ACBP=A9
 0001:0000381C 0000000E C=CODE     S=.text    G=(none)   M=PCEGlobs ACBP=A9
 0001:0000382C 0000000E C=CODE     S=.text    G=(none)   M=PakCust  ACBP=A9
 0001:0000383C 0000000E C=CODE     S=.text    G=(none)   M=PkgDir   ACBP=A9
 0001:0000384C 0000000E C=CODE     S=.text    G=(none)   M=PakComp  ACBP=A9
 0001:0000385C 0000000E C=CODE     S=.text    G=(none)   M=FileHist ACBP=A9
 0001:0000386C 0000000E C=CODE     S=.text    G=(none)   M=ProjectItem ACBP=A9
 0001:0000387C 0000000E C=CODE     S=.text    G=(none)   M=PrefOptDlg ACBP=A9
 0001:0000388C 0000000E C=CODE     S=.text    G=(none)   M=ReposCfg ACBP=A9
 0001:0000389C 0000000E C=CODE     S=.text    G=(none)   M=EditTpl  ACBP=A9
 0001:000038AC 0000000E C=CODE     S=.text    G=(none)   M=Template ACBP=A9
 0001:000038BC 0000000E C=CODE     S=.text    G=(none)   M=PrjTpl   ACBP=A9
 0001:000038CC 0000000E C=CODE     S=.text    G=(none)   M=FormTpl  ACBP=A9
 0001:000038DC 0000000E C=CODE     S=.text    G=(none)   M=PalEdit  ACBP=A9
 0001:000038EC 0000000E C=CODE     S=.text    G=(none)   M=GalBrow  ACBP=A9
 0001:000038FC 0000000E C=CODE     S=.text    G=(none)   M=ExptMain ACBP=A9
 0001:0000390C 0000000E C=CODE     S=.text    G=(none)   M=ParserThread ACBP=A9
 0001:0000391C 0000000E C=CODE     S=.text    G=(none)   M=EditMain ACBP=A9
 0001:0000392C 0000000E C=CODE     S=.text    G=(none)   M=VcsMain  ACBP=A9
 0001:0000393C 0000000E C=CODE     S=.text    G=(none)   M=VcsIntf  ACBP=A9
 0001:0000394C 0000000E C=CODE     S=.text    G=(none)   M=NewFile  ACBP=A9
 0001:0000395C 0000000E C=CODE     S=.text    G=(none)   M=DebugFindFile ACBP=A9
 0001:0000396C 0000000E C=CODE     S=.text    G=(none)   M=DataBPModify ACBP=A9
 0001:0000397C 0000000E C=CODE     S=.text    G=(none)   M=DataBPAdd ACBP=A9
 0001:0000398C 0000000E C=CODE     S=.text    G=(none)   M=AdrBPAdd ACBP=A9
 0001:0000399C 0000000E C=CODE     S=.text    G=(none)   M=BPModify ACBP=A9
 0001:000039AC 0000000E C=CODE     S=.text    G=(none)   M=BPAdd    ACBP=A9
 0001:000039BC 0000000E C=CODE     S=.text    G=(none)   M=WinMsg   ACBP=A9
 0001:000039CC 0000000E C=CODE     S=.text    G=(none)   M=AdrBPModify ACBP=A9
 0001:000039DC 0000000E C=CODE     S=.text    G=(none)   M=GetAddr  ACBP=A9
 0001:000039EC 0000000E C=CODE     S=.text    G=(none)   M=DisView  ACBP=A9
 0001:000039FC 0000000E C=CODE     S=.text    G=(none)   M=DisComp  ACBP=A9
 0001:00003A0C 0000000E C=CODE     S=.text    G=(none)   M=SelectTh ACBP=A9
 0001:00003A1C 0000000E C=CODE     S=.text    G=(none)   M=EdScript ACBP=A9
 0001:00003A2C 0000000E C=CODE     S=.text    G=(none)   M=GotoLine ACBP=A9
 0001:00003A3C 0000000E C=CODE     S=.text    G=(none)   M=VClient  ACBP=A9
 0001:00003A4C 0000000E C=CODE     S=.text    G=(none)   M=SrchPrgs ACBP=A9
 0001:00003A5C 0000000E C=CODE     S=.text    G=(none)   M=SrchDlg  ACBP=A9
 0001:00003A6C 0000000E C=CODE     S=.text    G=(none)   M=WinList  ACBP=A9
 0001:00003A7C 0000000E C=CODE     S=.text    G=(none)   M=BarFrm   ACBP=A9
 0001:00003A8C 0000000E C=CODE     S=.text    G=(none)   M=BottomBarFrm ACBP=A9
 0001:00003A9C 0000000E C=CODE     S=.text    G=(none)   M=RightBarFrm ACBP=A9
 0001:00003AAC 0000000E C=CODE     S=.text    G=(none)   M=LeftBarFrm ACBP=A9
 0001:00003ABC 0000000E C=CODE     S=.text    G=(none)   M=MainWorkFrm ACBP=A9
 0001:00003ACC 0000000E C=CODE     S=.text    G=(none)   M=WorkFrm  ACBP=A9
 0001:00003ADC 0000000E C=CODE     S=.text    G=(none)   M=PrintSes ACBP=A9
 0001:00003AEC 0000000E C=CODE     S=.text    G=(none)   M=PrintSts ACBP=A9
 0001:00003AFC 0000000E C=CODE     S=.text    G=(none)   M=OptStr   ACBP=A9
 0001:00003B0C 0000000E C=CODE     S=.text    G=(none)   M=RplcDlg  ACBP=A9
 0001:00003B1C 0000000E C=CODE     S=.text    G=(none)   M=FileMain ACBP=A9
 0001:00003B2C 0000000E C=CODE     S=.text    G=(none)   M=EdToken  ACBP=A9
 0001:00003B3C 0000000E C=CODE     S=.text    G=(none)   M=WorkspaceCrtrs ACBP=A9
 0001:00003B4C 000005A4 C=CODE     S=.text    G=(none)   M=MsgCmd   ACBP=A9
 0001:000040F0 00001828 C=CODE     S=.text    G=(none)   M=AddlCompInfFrm ACBP=A9
 0001:00005918 00000A2D C=CODE     S=.text    G=(none)   M=MsgInfo  ACBP=A9
 0002:00000000 0000002C C=DATA     S=.data    G=DGROUP   M=SysInit  ACBP=A9
 0002:0000002C 00000002 C=DATA     S=.data    G=DGROUP   M=RegExpComp ACBP=A9
 0002:00000030 000000BC C=DATA     S=.data    G=DGROUP   M=AddlCompInfFrm ACBP=A9
 0002:00001000 00000010 C=BSS      S=.bss     G=DGROUP   M=SysInit  ACBP=A9
 0002:00001010 00000004 C=BSS      S=.bss     G=DGROUP   M=Windows  ACBP=A9
 0002:00001014 00000004 C=BSS      S=.bss     G=DGROUP   M=Messages ACBP=A9
 0002:00001018 00000004 C=BSS      S=.bss     G=DGROUP   M=CommCtrl ACBP=A9
 0002:0000101C 00000004 C=BSS      S=.bss     G=DGROUP   M=Imm      ACBP=A9
 0002:00001020 00000004 C=BSS      S=.bss     G=DGROUP   M=ShlObj   ACBP=A9
 0002:00001024 00000004 C=BSS      S=.bss     G=DGROUP   M=UrlMon   ACBP=A9
 0002:00001028 00000004 C=BSS      S=.bss     G=DGROUP   M=WinInet  ACBP=A9
 0002:0000102C 00000004 C=BSS      S=.bss     G=DGROUP   M=RegStr   ACBP=A9
 0002:00001030 00000004 C=BSS      S=.bss     G=DGROUP   M=ShellAPI ACBP=A9
 0002:00001034 00000004 C=BSS      S=.bss     G=DGROUP   M=WinSpool ACBP=A9
 0002:00001038 00000004 C=BSS      S=.bss     G=DGROUP   M=CommDlg  ACBP=A9
 0002:0000103C 00000004 C=BSS      S=.bss     G=DGROUP   M=Dlgs     ACBP=A9
 0002:00001040 00000004 C=BSS      S=.bss     G=DGROUP   M=RichEdit ACBP=A9
 0002:00001044 00000004 C=BSS      S=.bss     G=DGROUP   M=RegExpConst ACBP=A9
 0002:00001048 00000004 C=BSS      S=.bss     G=DGROUP   M=RegExpComp ACBP=A9
 0002:0000104C 00000004 C=BSS      S=.bss     G=DGROUP   M=MMSystem ACBP=A9
 0002:00001050 00000008 C=BSS      S=.bss     G=DGROUP   M=MsgCmd   ACBP=A9
 0002:00001058 0000001C C=BSS      S=.bss     G=DGROUP   M=AddlCompInfFrm ACBP=A9


  Address         Publics by Name

 0002:00001008       .1
 0002:0000102C       .1
 0002:00001014       .1
 0002:0000103C       .1
 0002:00001028       .1
 0002:00001040       .1
 0002:00001038       .1
 0002:00001024       .1
 0002:00001044       .1
 0002:00001018       .1
 0002:00001020       .1
 0002:00001030       .1
 0002:0000101C       .1
 0002:00001010       .3
 0002:00001034       .3
 0002:00001054       .3
 0002:0000105C       .3
 0002:00001048       .5
 0002:0000104C       .7
 0001:00006320       @GetPackageInfoTable
 0001:000002D0       @InitPkg
 0001:00006328       @PackageLoad
 0001:00000334       @PackageLoad
 0001:00000340       @PackageUnload
 0001:00006334       @PackageUnload
 0001:00003EFC       AddActionMenu
 0001:00005240       AddHint
 0001:000058B8       AddlCompInfFrm
 0001:000001D0       AllocTlsBuffer
 0001:00000794       CommCtrl
 0001:00000B8C       CommDlg
 0001:00000BC4       Dlgs
 0001:0000038C       DrawFocusRect
 0001:00000394       DrawText
 0001:0000027C       ExitProcessTLS
 0001:00000254       ExitThreadTLS
 0001:00000A24       Finalization
 0001:00002C64       Finalization
 0001:000009EC       Finalization
 0001:000009B4       Finalization
 0001:0000097C       Finalization
 0001:000008D4       Finalization
 0001:00000764       Finalization
 0001:00000A64       Finalization
 0001:0000039C       Finalization
 0001:00002B64       Finalization
 0001:000040AC       Finalization
 0001:0000034C       Finalization
 0001:00000B24       Finalization
 0001:00000B5C       Finalization
 0001:00000B94       Finalization
 0001:00005860       Finalization
 0001:00000C1C       Finalization
 0001:000003E4       Finalization
 0001:00000E84       Finalization
 0001:00000198       FreeLibrary
 0001:00000384       GetModuleFileName
 0001:000001DC       GetTlsSize
 0002:00001004       HInstance
 0001:00004098       IDERegister
 0001:00000904       Imm
 0001:000002A0       InitializeModule
 0001:00000228       InitProcessTLS
 0001:000001E4       InitThreadTLS
 0001:000001A0       LocalAlloc
 0001:000001A8       LocalFree
 0001:00000414       Messages
 0001:00002C94       MMSystem
 0002:00000004       Module
 0002:00001000       ModuleIsLib
 0002:00001001       ModuleIsPackage
 0001:000040E8       MsgCmd
 0002:00001058       MsgHook
 0001:00006340       MsgInfo
 0002:00000030       Msgs
 0002:00001060       Notifier
 0001:00005360       ProcessSection
 0002:00001050       ProductStartup
 0001:0000134C       REError
 0001:00002B94       RegExpComp
 0001:00000EB4       RegExpConst
 0001:00000A54       RegStr
 0001:00000C4C       RichEdit
 0002:0000106C       sError
 0002:00001070       sFatalError
 0001:00000A94       ShellAPI
 0001:00000A5C       ShellExecute
 0002:00001064       sHint
 0001:000009AC       ShlObj
 0001:00001364       StrCSpan
 0002:00001068       sWarning
 0001:0000037C       SysInit
 0001:00001CC0       TCompiledRE.CharOpnd
 0001:00001924       TCompiledRE.Create
 0001:00001A9C       TCompiledRE.Destroy
 0001:00001B10       TCompiledRE.EmitBlankSet
 0001:00001AC0       TCompiledRE.EmitChar
 0001:00001B58       TCompiledRE.EmitCharSet
 0001:00001AD8       TCompiledRE.EmitCopy
 0001:00001C08       TCompiledRE.EmitInsert
 0001:00001AEC       TCompiledRE.EmitNode
 0001:00001C6C       TCompiledRE.EmitOpndTailFixup
 0001:00001C3C       TCompiledRE.EmitTailFixup
 0001:0000253C       TCompiledRE.Match
 0001:000027E0       TCompiledRE.MatchExec
 0001:00002704       TCompiledRE.MatchSimpleCount
 0001:000026D0       TCompiledRE.MatchText
 0001:00001CA0       TCompiledRE.NextNode
 0001:00001CB8       TCompiledRE.NodeOpnd
 0001:00002160       TCompiledRE.ScanAtom
 0001:00001EC0       TCompiledRE.ScanBranch
 0001:00001F4C       TCompiledRE.ScanPiece
 0001:00001CC8       TCompiledRE.ScanRE
 0001:000001B0       TlsAlloc
 0002:0000100C       tlsBuffer
 0001:000001B8       TlsFree
 0001:000001C0       TlsGetValue
 0002:00000000       TlsIndex
 0002:D8FF8000       TlsLast
 0002:0000001C       TlsProc
 0001:000001C8       TlsSetValue
 0001:0000552C       TMessageHintFrm.AfterCompile
 0001:00005808       TMessageHintFrm.AfterSave
 0001:00005798       TMessageHintFrm.BeforeCompile
 0001:0000580C       TMessageHintFrm.BeforeSave
 0001:00004B8C       TMessageHintFrm.ClearActnExecute
 0001:00004C50       TMessageHintFrm.CopyAllExecute
 0001:00004BE8       TMessageHintFrm.CopyMsgExecute
 0001:00004CAC       TMessageHintFrm.CopyMsgUpdate
 0001:000046C8       TMessageHintFrm.Destroy
 0001:00005810       TMessageHintFrm.Destroyed
 0001:000051A0       TMessageHintFrm.DownLoadURL1DownloadProgress
 0001:00005800       TMessageHintFrm.FileNotification
 0001:00004768       TMessageHintFrm.FormCreate
 0001:00005844       TMessageHintFrm.FormDestroy
 0001:00005008       TMessageHintFrm.FormResize
 0001:00004F70       TMessageHintFrm.MessagesListClick
 0001:00004CE0       TMessageHintFrm.MessagesListDblClick
 0001:00004DA0       TMessageHintFrm.MessagesListDrawItem
 0001:00005014       TMessageHintFrm.MessagesListKeyDown
 0001:00005814       TMessageHintFrm.Modified
 0001:00004BAC       TMessageHintFrm.ViewMsgFileExecute
 0001:00003DB0       TMsgInfoCommands.ProSkuCommandsCreate
 0001:00003DE0       TMsgInfoCommands.ProSkuCommandsDestroy
 0001:00003DF0       TMsgInfoCommands.ViewAddlMsgInfoCommandExecute
 0001:00005818       TMsgNotifier.EventNotification
 0001:0000583C       TMsgNotifier.FileNotification
 0001:00003E1C       TProductStartup.Create
 0001:00003E64       TProductStartup.Destroy
 0001:00003EA8       TProductStartup.Notification
 0001:00003FA0       TProductStartup.ProductStartup
 0001:0000188C       TRegularExpression.Compile
 0001:00001384       TRegularExpression.Create
 0001:000013C4       TRegularExpression.CreateRE
 0001:00001410       TRegularExpression.Destroy
 0001:0000146C       TRegularExpression.GetCharCount
 0001:00001474       TRegularExpression.GetCharSet
 0001:00001880       TRegularExpression.GetCompiled
 0001:0000157C       TRegularExpression.GetIsMatch
 0001:000015BC       TRegularExpression.GetMatch
 0001:000015A8       TRegularExpression.GetMatchCount
 0001:00001808       TRegularExpression.GetMatchLen
 0001:00001794       TRegularExpression.GetMatchPos
 0001:000018E4       TRegularExpression.Match
 0001:000014F4       TRegularExpression.ResetMatches
 0001:00001490       TRegularExpression.SetCharSet
 0001:0000163C       TRegularExpression.SetMatch
 0001:00001524       TRegularExpression.SetPattern
 0001:0000143C       TRegularExpression.SetREOptions
 0001:00001550       TRegularExpression.SetText
 0001:000018C4       TRegularExpression.UnCompile
 0001:000002AC       UninitializeModule
 0001:000009E4       UrlMon
 0002:0000002C       WhichAny
 0001:000003CC       Windows
 0001:00000A1C       WinInet
 0001:00000B54       WinSpool


  Address         Publics by Value

 0002:D8FF8000       TlsLast
 0001:00000198       FreeLibrary
 0001:000001A0       LocalAlloc
 0001:000001A8       LocalFree
 0001:000001B0       TlsAlloc
 0001:000001B8       TlsFree
 0001:000001C0       TlsGetValue
 0001:000001C8       TlsSetValue
 0001:000001D0       AllocTlsBuffer
 0001:000001DC       GetTlsSize
 0001:000001E4       InitThreadTLS
 0001:00000228       InitProcessTLS
 0001:00000254       ExitThreadTLS
 0001:0000027C       ExitProcessTLS
 0001:000002A0       InitializeModule
 0001:000002AC       UninitializeModule
 0001:000002D0       @InitPkg
 0001:00000334       @PackageLoad
 0001:00000340       @PackageUnload
 0001:0000034C       Finalization
 0001:0000037C       SysInit
 0001:00000384       GetModuleFileName
 0001:0000038C       DrawFocusRect
 0001:00000394       DrawText
 0001:0000039C       Finalization
 0001:000003CC       Windows
 0001:000003E4       Finalization
 0001:00000414       Messages
 0001:00000764       Finalization
 0001:00000794       CommCtrl
 0001:000008D4       Finalization
 0001:00000904       Imm
 0001:0000097C       Finalization
 0001:000009AC       ShlObj
 0001:000009B4       Finalization
 0001:000009E4       UrlMon
 0001:000009EC       Finalization
 0001:00000A1C       WinInet
 0001:00000A24       Finalization
 0001:00000A54       RegStr
 0001:00000A5C       ShellExecute
 0001:00000A64       Finalization
 0001:00000A94       ShellAPI
 0001:00000B24       Finalization
 0001:00000B54       WinSpool
 0001:00000B5C       Finalization
 0001:00000B8C       CommDlg
 0001:00000B94       Finalization
 0001:00000BC4       Dlgs
 0001:00000C1C       Finalization
 0001:00000C4C       RichEdit
 0001:00000E84       Finalization
 0001:00000EB4       RegExpConst
 0001:0000134C       REError
 0001:00001364       StrCSpan
 0001:00001384       TRegularExpression.Create
 0001:000013C4       TRegularExpression.CreateRE
 0001:00001410       TRegularExpression.Destroy
 0001:0000143C       TRegularExpression.SetREOptions
 0001:0000146C       TRegularExpression.GetCharCount
 0001:00001474       TRegularExpression.GetCharSet
 0001:00001490       TRegularExpression.SetCharSet
 0001:000014F4       TRegularExpression.ResetMatches
 0001:00001524       TRegularExpression.SetPattern
 0001:00001550       TRegularExpression.SetText
 0001:0000157C       TRegularExpression.GetIsMatch
 0001:000015A8       TRegularExpression.GetMatchCount
 0001:000015BC       TRegularExpression.GetMatch
 0001:0000163C       TRegularExpression.SetMatch
 0001:00001794       TRegularExpression.GetMatchPos
 0001:00001808       TRegularExpression.GetMatchLen
 0001:00001880       TRegularExpression.GetCompiled
 0001:0000188C       TRegularExpression.Compile
 0001:000018C4       TRegularExpression.UnCompile
 0001:000018E4       TRegularExpression.Match
 0001:00001924       TCompiledRE.Create
 0001:00001A9C       TCompiledRE.Destroy
 0001:00001AC0       TCompiledRE.EmitChar
 0001:00001AD8       TCompiledRE.EmitCopy
 0001:00001AEC       TCompiledRE.EmitNode
 0001:00001B10       TCompiledRE.EmitBlankSet
 0001:00001B58       TCompiledRE.EmitCharSet
 0001:00001C08       TCompiledRE.EmitInsert
 0001:00001C3C       TCompiledRE.EmitTailFixup
 0001:00001C6C       TCompiledRE.EmitOpndTailFixup
 0001:00001CA0       TCompiledRE.NextNode
 0001:00001CB8       TCompiledRE.NodeOpnd
 0001:00001CC0       TCompiledRE.CharOpnd
 0001:00001CC8       TCompiledRE.ScanRE
 0001:00001EC0       TCompiledRE.ScanBranch
 0001:00001F4C       TCompiledRE.ScanPiece
 0001:00002160       TCompiledRE.ScanAtom
 0001:0000253C       TCompiledRE.Match
 0001:000026D0       TCompiledRE.MatchText
 0001:00002704       TCompiledRE.MatchSimpleCount
 0001:000027E0       TCompiledRE.MatchExec
 0001:00002B64       Finalization
 0001:00002B94       RegExpComp
 0001:00002C64       Finalization
 0001:00002C94       MMSystem
 0001:00003DB0       TMsgInfoCommands.ProSkuCommandsCreate
 0001:00003DE0       TMsgInfoCommands.ProSkuCommandsDestroy
 0001:00003DF0       TMsgInfoCommands.ViewAddlMsgInfoCommandExecute
 0001:00003E1C       TProductStartup.Create
 0001:00003E64       TProductStartup.Destroy
 0001:00003EA8       TProductStartup.Notification
 0001:00003EFC       AddActionMenu
 0001:00003FA0       TProductStartup.ProductStartup
 0001:00004098       IDERegister
 0001:000040AC       Finalization
 0001:000040E8       MsgCmd
 0001:000046C8       TMessageHintFrm.Destroy
 0001:00004768       TMessageHintFrm.FormCreate
 0001:00004B8C       TMessageHintFrm.ClearActnExecute
 0001:00004BAC       TMessageHintFrm.ViewMsgFileExecute
 0001:00004BE8       TMessageHintFrm.CopyMsgExecute
 0001:00004C50       TMessageHintFrm.CopyAllExecute
 0001:00004CAC       TMessageHintFrm.CopyMsgUpdate
 0001:00004CE0       TMessageHintFrm.MessagesListDblClick
 0001:00004DA0       TMessageHintFrm.MessagesListDrawItem
 0001:00004F70       TMessageHintFrm.MessagesListClick
 0001:00005008       TMessageHintFrm.FormResize
 0001:00005014       TMessageHintFrm.MessagesListKeyDown
 0001:000051A0       TMessageHintFrm.DownLoadURL1DownloadProgress
 0001:00005240       AddHint
 0001:00005360       ProcessSection
 0001:0000552C       TMessageHintFrm.AfterCompile
 0001:00005798       TMessageHintFrm.BeforeCompile
 0001:00005800       TMessageHintFrm.FileNotification
 0001:00005808       TMessageHintFrm.AfterSave
 0001:0000580C       TMessageHintFrm.BeforeSave
 0001:00005810       TMessageHintFrm.Destroyed
 0001:00005814       TMessageHintFrm.Modified
 0001:00005818       TMsgNotifier.EventNotification
 0001:0000583C       TMsgNotifier.FileNotification
 0001:00005844       TMessageHintFrm.FormDestroy
 0001:00005860       Finalization
 0001:000058B8       AddlCompInfFrm
 0001:00006320       @GetPackageInfoTable
 0001:00006328       @PackageLoad
 0001:00006334       @PackageUnload
 0001:00006340       MsgInfo
 0002:00000000       TlsIndex
 0002:00000004       Module
 0002:0000001C       TlsProc
 0002:0000002C       WhichAny
 0002:00000030       Msgs
 0002:00001000       ModuleIsLib
 0002:00001001       ModuleIsPackage
 0002:00001004       HInstance
 0002:00001008       .1
 0002:0000100C       tlsBuffer
 0002:00001010       .3
 0002:00001014       .1
 0002:00001018       .1
 0002:0000101C       .1
 0002:00001020       .1
 0002:00001024       .1
 0002:00001028       .1
 0002:0000102C       .1
 0002:00001030       .1
 0002:00001034       .3
 0002:00001038       .1
 0002:0000103C       .1
 0002:00001040       .1
 0002:00001044       .1
 0002:00001048       .5
 0002:0000104C       .7
 0002:00001050       ProductStartup
 0002:00001054       .3
 0002:00001058       MsgHook
 0002:0000105C       .3
 0002:00001060       Notifier
 0002:00001064       sHint
 0002:00001068       sWarning
 0002:0000106C       sError
 0002:00001070       sFatalError


Bound resource files

MsgCmd.dfm
AddlCompInfFrm.dfm
MsgInfo.res
C:\DOCUME~1\~KOKOP~1\LOCALS~1\Temp\dtf285A.tmp


Program entry point at 0001:00006340
